:100000008328FF3FFF3FFF3F0000031383169C1C24
:100010000B28000005288312370883169B008312E3
:10002000380883169A009C131C158B1355309D00BD
:10003000AA309D009C148B171C110800A5300313D7
:100040008312FA00FA0B22280000000008000313B4
:100050008312320883169B009C131C141A08F000AC
:10006000080003138312B7012008B800042082306F
:10007000FB00FF30FA00FB0B3E284128FA0B3E281C
:100080003B288730FA00FA0B4328000008000313CE
:1000900083123308F0000130F100F20170080319F7
:1000A0005628F10DF20D7110FF3F4F287108B60070
:1000B000320884000008F0007108F0057008013073
:1000C000031D0030F0003508F006031981283408BC
:1000D000003C03186F281E201E20B4036728320836
:1000E00084000008F0003608F00570080130031D98
:1000F0000030F0003508F00603198128FF30F000C9
:100100000800F00108000730031383129F0010302D
:1001100083168500860183128601A1013F30A2006B
:100120000630A3005B30A4004F30A5006630A60067
:100130006D30A7007D30A8000730A9007F30AA00ED
:100140006F30AB007730AC007C30AD003930AE00A2
:100150005E30AF007930B0007130B100B2012720BD
:1001600070088312A0008230FB00FF30FA00FB0B06
:10017000BA28BD28FA0BBA28B7288730FA00FA0B3C
:10018000BF28000020080F3C0318C828A001312018
:1001900083122008223F84000008860001302005D9
:1001A000F000003070180130050601398506003076
:1001B000A0180130F1000030711802300506023934
:1001C0008506003020190130F1000030711804302C
:1001D0000506043985060030A0190130F100003011
:1001E000711808300506083985060530B20004305C
:1001F000B3000130B400B50147207008031902298B
:100200000130A1002108031915290530B20004307E
:10021000B3000130B4000130B50047207008031965
:100220001529A00A31208312A101AE281629FF3F0B
:02400E00583F19
:00000001FF
